:100000000C946B010C9488010C9488010C94880169
:100010000C9491080C949D070C9464080C940A08A5
:100020000C9437080C9470070C94DD070C941D0792
:100030000C9488010C9423030C9488010C94EC021A
:100040000C940A090C9488010C9488010C94880182
:100050000C948801303132333435363738394142E7
:100060004344454600000001000800200040008095
:100070000000010004000001000800400000010031
:10008000041B63001B5B324A001B5B25646D001B75
:100090005B3F323568001B5B3F32356C001B5B25D4
:1000A000643B25644800636F6D6D616E64206E6F04
:1000B0007420666F756E6400636D646C696E653A7A
:1000C0002000633E0079A780E3888D90AB9946A21B
:1000D00063AC0BB646C11CCC98D8C3E5A680858B13
:1000E00091989EA5ADB5BDC5CEE7E0EAF580008646
:1000F000478C8B92C798F89F19A527AB1EB0FBB60B
:10010000B9BC56C1CDC71CCC3FD133D5F4DA81DEA2
:10011000D6E2F1E6CEEA6CEDC9F0E1F3B5F640F8CF
:1001200083FA7CFC29FD89FE9CFF61FFD7FFFEFF5F
:10013000D7FF61FE9CFD89FC29FA7CF883F640F329
:10014000B5F0E1EDC9EA6CE6CEE2F1DED6DA81D5B2
:10015000F5D133CC3FC71CC1CDBC56B6B9B0FBAB53
:100160001EA5279F1998F892C78C8B864780007927
:10017000B873746D38670760E65AD854E14F044984
:100180004643A93E3238E333C02ECC2A0B257E21CC
:10019000291D0E1931159312360F1E0C4B09BF077E
:1001A0007C058303D702760163009E0028000100CE
:1001B00028009E0163027603D60583077C09BF0CE5
:1001C0004A0F1E1236159319311D0E2129257E2A3C
:1001D0000A2ECC33C038E33E3243A949464F04547B
:1001E000E05AD860E667076D37737479B845656C77
:1001F00020636F6D6D616E647A210D0A0045786928
:100200007465642070726F6772616D210D0A00253C
:1002100064202020256420002564202020256420DF
:100220000D0A00696E702076616C203D2025640DFA
:100230000A006B6579626F617264576F7264313A5C
:10024000202025640D0A00696E6465783A2020201C
:100250002020202020202025640D0A007068617372
:100260006544656C74613A202020202025640D0AC5
:1002700000696E702076616C203D20256420200D81
:100280000A0025640D0A0025640D0A000D0A000D00
:100290000A002825642920256420202020000D0A3A
:1002A000000D0A57656C636F6D6520746F2045788B
:1002B000657274696F6E20496E737472756D656EC8
:1002C00074206261636B646F6F72210D0A00256494
:1002D00020000D0A000011241FBECFE5D8E0DEBFCC
:1002E000CDBF11E0A0E6B0E0ECE0F8E202C005907E
:1002F0000D92A83CB107D9F717E0A8ECB1E001C016
:100300001D92A83DB107E1F70E945C100C94051402
:100310000C940000FC019A014FB7F894718360833C
:100320003383228317821682158214824FBF089569
:10033000CF93DF93DC01E0E06FB7F894EC014C81E0
:100340005D8141155105C9F0ED91FC9111978E81A8
:100350009F81E80FF91FE08101969F838E832A8198
:100360003B818217930720F0821B930B9F838E8320
:1003700041505040ED015D834C836FBF8E2F992714
:10038000DF91CF910895FC01AFB7F8944481558176
:1003900064177507A0F486819781860F971F97834E
:1003A0008683228133818217930720F0821B930B6F
:1003B00097838683461B570B5583448302C015825F
:1003C0001482AFBF08951F93FC011FB7F894868174
:1003D000978122813381860F971FB9010E94721382
:1003E0000190F081E02DE80FF91F80811FBF992750
:1003F0001F9108951F93CF93DF93EC01162F4FB7F2
:10040000F8942C813D816A817B8126173707A0F4FF
:100410008E819F81820F931F0E947213E881F98160
:10042000E80FF91F10838C819D8101969D838C8339
:100430004FBF8FEF90E003C04FBF80E090E0DF91AF
:10044000CF911F910895FC014FB7F8942281338119
:10045000848195814FBF281B390BC9010895FC0188
:100460008FB7F894158214828FBF0895DC01CB01F9
:1004700073E0880F991FAA1FBB1F7A95D1F79C01C3
:10048000AD01220F331F441F551F80509C4DAB40C0
:10049000BF4FBC01CD010E948613DA01C90101974B
:1004A00089B9892F992780BD089540E450E068EC10
:1004B00071E081E595E00E948A0140E450E068E047
:1004C00072E08AE595E00E948A0108950E94550233
:1004D000109249021092480288ED8AB960E875E2EC
:1004E00080E090E00E9436028FEF809350051092DA
:1004F00059051092630510926205789408959093BF
:10050000490280934802089581E595E008958AE5BF
:1005100095E00895982F809150058823E1F39CB9C8
:10052000109250050895CF93DF93EC01809153050D
:1005300090915405009769F080915505909156056A
:10054000009739F081E595E00E94980188838FEF4C
:1005500090E0DF91CF910895CF93DF93CDB7DEB7D1
:1005600021970FB6F894DEBF0FBECDBFCE01019626
:100570000E949302882319F08981992702C08FEF86
:100580009FEF21960FB6F894DEBF0FBECDBFDF916F
:10059000CF910895109256051092550508958091B7
:1005A000550590915605892B19F48FEF90E0089529
:1005B00080E090E00895682F8AE595E00E94FA01B6
:1005C000992708958FEF809359058AE595E00E9459
:1005D00098010E948A0208951F920F920FB60F92FF
:1005E00011242F933F934F935F936F937F938F9338
:1005F0009F93AF93BF93EF93FF9380915905882307
:1006000071F080915E0590915F05892B31F08AE54C
:1006100095E00E9498018CB905C0109259058FEFA2
:1006200080935005FF91EF91BF91AF919F918F9172
:100630007F916F915F914F913F912F910F900FBEDE
:100640000F901F9018951F920F920FB60F921124C2
:100650002F933F934F935F936F937F938F939F93CA
:10066000AF93BF93EF93FF936CB180914802909149
:100670004902892B39F0E0914802F0914902862F16
:1006800009950FC081E595E00E94FA01882349F49D
:100690008091620590916305019690936305809324
:1006A0006205FF91EF91BF91AF919F918F917F91E3
:1006B0006F915F914F913F912F910F900FBE0F90CF
:1006C0001F90189590934B0280934A020895CF9300
:1006D000C82F8A3031F4E0914A02F0914B028DE04C
:1006E0000995E0914A02F0914B028C2F0995CF9128
:1006F0000895CF93DF93EC01892B49F088818823FB
:1007000031F089910E94670388818823D1F7DF91B6
:10071000CF910895EF92FF920F931F93CF93DF93A2
:100720008C017A01C0E0D0E0892BE9F0CE0121965E
:100730008617970728F4F80181918F018823B1F774
:10074000C0E0D0E0CE15DF0570F4F8018081882389
:1007500019F00F5F1F4F01C080E20E9467032196CE
:10076000CE15DF0590F3DF91CF911F910F91FF9090
:10077000EF900895CF93DF93EC01009761F0FC01B7
:1007800021968491882339F00E946703FE01219607
:1007900084918823C9F7DF91CF9108958AE00E9460
:1007A00067030895E82FFF27EF70F070EC5AFF4FB2
:1007B00084910E94670308951F93182F82958F706C
:1007C0000E94D203812F0E94D2031F9108950F939C
:1007D0001F938C01812F99270E94DC03802F0E9498
:1007E000DC031F910F910895EF92FF920F931F93D7
:1007F0007B018C01C801AA27BB270E94E703C70120
:100800000E94E7031F910F91FF90EF9008952F92A0
:100810003F924F925F926F927F928F929F92AF9290
:10082000BF92CF92DF92EF92FF920F931F93CF93DD
:10083000DF93CDB7DEB7A2970FB6F894DEBF0FBE39
:10084000CDBF69A3242E2AA337014801442351F0C8
:1008500017FF08C0EE24FF248701E618F7080809EF
:10086000190902C08401730199A1692F772767FDD7
:10087000709561507040222011F061507040362E0A
:1008800018A22FE1422E512C4C0E5D1EA82EBB2427
:10089000A7FCB094CB2CDB2CC801B701A6019501B5
:1008A0000E948613DC01CB01FC01EF70F070EC5A62
:1008B000FF4F84918F8FC801B701A60195010E9457
:1008C000861379018A013A94EFEF3E1649F1C2018D
:1008D0000197E114F10401051105D1F02C01C801C3
:1008E000B701A60195010E948613DC01CB01FC0132
:1008F000EF70F070EC5AFF4F8491F2018083C801D1
:10090000B701A60195010E94861379018A0104C0EE
:100910002C018AA1F20180833A949FEF3916B9F62F
:100920002220A9F097FE05C08DE2F20182932F01EB
:100930000EC0C201019716141704180419041CF400
:100940002C018BE202C02C0180E2F201808339A0ED
:100950003A94FFEF3F1649F0F20181912F010E9476
:1009600067033A94FFEF3F16B9F7A2960FB6F894D3
:10097000DEBF0FBECDBFDF91CF911F910F91FF90D2
:10098000EF90DF90CF90BF90AF909F908F907F902F
:100990006F905F904F903F902F9008957F928F922D
:1009A0009F92AF92BF92CF92DF92EF92FF920F93FE
:1009B0001F93CF93DF93CDB7DEB77888C988DA88E5
:1009C00073E1A72EB12CAC0EBD1E05C0882309F41F
:1009D00077C00E94670396012F5F3F4F772021F079
:1009E000F6016901849103C0F601808169018532B5
:1009F00069F72F5F3F4F772021F0F601690184915D
:100A000003C0F60180816901282F332727FD309527
:100A10002436310591F02536310524F4233631058D
:100A200029F0D7CF2837310581F0D3CFF50122E067
:100A300030E0A20EB31E8081CCCF6AE0862E912CCE
:100A400050E1E52E57E2F52E06C040E1842E912CB0
:100A5000E12C30E1F32EF50122E030E0A20EB31ECE
:100A6000008111818436C1F417FF06C010950195ED
:100A70001F4F8DE20E94670332E0E316F10460F03D
:100A80000E151F0548F4C7016AE070E00E9472135A
:100A90007B0162307105A0F7C801B7010E94721393
:100AA000CB010E94D203C801B7010E9472138C01CE
:100AB000C701B4010E9472137B01672B69F78BCFCA
:100AC00080E090E0DF91CF911F910F91FF90EF9028
:100AD000DF90CF90BF90AF909F908F907F900895C0
:100AE000039665E070E00E947213CB01AA27BB2732
:100AF00024E0880F991FAA1FBB1F2A95D1F720E079
:100B000030E02817390718F42F5F3F4FFACF0895C8
:100B1000883040F4E82FFF27EE0FFF1FE45BFD4F06
:100B200011821082089593B7987F982B93BF0895F0
:100B30001092640510926505109266051092670583
:100B4000089582E00E94930512BE89B7816089BF33
:100B50000E94980508959EB5987F982B9EBD089594
:100B600083E00E94AB051DBC1CBC89B7846089BFB3
:100B7000089595B5987F982B95BD089510926C05B2
:100B800010926D0510926E0510926F05089584E025
:100B90000E94B90514BC89B7806489BF0E94BE0554
:100BA0000895CF93C0E08C2F0E948805CF5FC83096
:100BB000D0F30E94A1050E94B0050E94C705789459
:100BC000CF91089583B7E82FFF27E770F070EE0FFD
:100BD000FF1FEB58FF4F8591949108958EB5E82F34
:100BE000FF27E770F070EE0FFF1FEB58FF4F859166
:100BF0009491089585B5E82FFF27E770F070EE0F08
:100C0000FF1FEB59FF4F859194910895883040F470
:100C1000E82FFF27EE0FFF1FE45BFD4F718360831A
:100C20000895DF92EF92FF920F931F93CF93DF937C
:100C3000EC01D2B6109268051092690510926A050F
:100C400010926B050E94E2059C014427552760E045
:100C500074E284EF90E00E94A813293B8DE83807E6
:100C600086E0480780E05807C0F487E2C131D80722
:100C7000A0F4CE01AA27BB27BC01CD010E945313CB
:100C8000DC01CB01BC01CD0128EE33E040E050E0B7
:100C90000E948613FA01E90111C07E010027112785
:100CA000CA01B90128EE33E040E050E00E9486130B
:100CB000C801B7010E945313FC01EB018091680544
:100CC00090916905A0916A05B0916B052227382F94
:100CD000492F5A2F82B79927AA27BB27282B392BB0
:100CE0004A2B5B2BCD0DD11DE11DF11D2C173D07AE
:100CF0004E075F0758F58091680590916905A091AE
:100D00006A05B0916B0585B78F7885BF85B7806818
:100D100085BF889585B78F7785BF8091680590914D
:100D20006905A0916A05B0916B05BA2FA92F982F7C
:100D3000882722B7332744275527822B932BA42BB0
:100D4000B52B8C179D07AE07BF07A8F2DF91CF9197
:100D50001F910F91FF90EF90DF90089580916405AF
:100D600090916505A0916605B0916705BC01CD0124
:100D7000089580916C0590916D05A0916E05B091DC
:100D80006F05BC01CD010895893031F48FB58260C3
:100D90008FBD8FB58E7F0AC08A3019F48FB58260FF
:100DA00002C08FB58D7F8FBD8FB581608FBD1BBC9D
:100DB0001ABC19BC18BC08959C018FB58E7F8FBDDD
:100DC0008FB582608FBD8EB588608EBD8EB5806117
:100DD0008EBD37BD26BD1BBC1ABC19BC18BC0895FE
:100DE0008FB58F778FBD8FB58F7B8FBD08958FB5F2
:100DF0008F7D8FBD8FB58F7E8FBD08958FB58D7F11
:100E00008FBD8FB58E7F8FBD0E94F0060E94F706C2
:100E100008958FB580688FBD8FB58F7B8FBD089586
:100E20008FB580628FBD8FB58F7E8FBD08959BBDBE
:100E30008ABD089599BD88BD08951F920F920FB67F
:100E40000F9211242F933F934F935F936F937F9350
:100E50008F939F93AF93BF93EF93FF93809164051C
:100E600090916505A0916605B09167050196A11D59
:100E7000B11D8093640590936505A0936605B093BA
:100E800067058091680590916905A0916A05B09108
:100E90006B050196A11DB11D8093680590936905AE
:100EA000A0936A05B0936B0580914C0290914D021E
:100EB000892B29F0E0914C02F0914D020995FF91A8
:100EC000EF91BF91AF919F918F917F916F915F91C2
:100ED0004F913F912F910F900FBE0F901F9018953B
:100EE0001F920F920FB60F9211242F933F934F939F
:100EF0005F936F937F938F939F93AF93BF93EF9382
:100F0000FF9380914E0290914F02892B29F0E0913E
:100F10004E02F0914F020995FF91EF91BF91AF9171
:100F20009F918F917F916F915F914F913F912F9101
:100F30000F900FBE0F901F9018951F920F920FB633
:100F40000F9211242F933F934F935F936F937F934F
:100F50008F939F93AF93BF93EF93FF9380916C0513
:100F600090916D05A0916E05B0916F050196A11D40
:100F7000B11D80936C0590936D05A0936E05B093A1
:100F80006F058091560290915702892B29F0E091CC
:100F90005602F09157020995FF91EF91BF91AF91E1
:100FA0009F918F917F916F915F914F913F912F9181
:100FB0000F900FBE0F901F9018951F920F920FB6B3
:100FC0000F9211242F933F934F935F936F937F93CF
:100FD0008F939F93AF93BF93EF93FF9380915A02A8
:100FE00090915B02892B29F0E0915A02F0915B020B
:100FF0000995FF91EF91BF91AF919F918F917F9153
:101000006F915F914F913F912F910F900FBE0F9075
:101010001F9018951F920F920FB60F9211242F93C5
:101020003F934F935F936F937F938F939F93AF9370
:10103000BF93EF93FF938091500290915102892BBF
:1010400029F0E0915002F09151020995FF91EF9142
:10105000BF91AF919F918F917F916F915F914F91D0
:101060003F912F910F900FBE0F901F9018951F92D8
:101070000F920FB60F9211242F933F934F935F93CC
:101080006F937F938F939F93AF93BF93EF93FF9350
:101090008091520290915302892B29F0E0915202E3
:1010A000F09153020995FF91EF91BF91AF919F91FC
:1010B0008F917F916F915F914F913F912F910F9001
:1010C0000FBE0F901F9018951F920F920FB60F92A0
:1010D00011242F933F934F935F936F937F938F933D
:1010E0009F93AF93BF93EF93FF938091540290919E
:1010F0005502892B29F0E0915402F091550209958F
:10110000FF91EF91BF91AF919F918F917F916F91DF
:101110005F914F913F912F910F900FBE0F901F90B5
:1011200018951F920F920FB60F9211242F933F9391
:101130004F935F936F937F938F939F93AF93BF93DF
:10114000EF93FF938091580290915902892B29F0D7
:10115000E0915802F09159020995FF91EF91BF91EA
:10116000AF919F918F917F916F915F914F913F913F
:101170002F910F900FBE0F901F90189596B1987FEA
:10118000982B96B9089527B12F73992736E0880FC9
:10119000991F3A95E1F7282B27B90895379A359882
:1011A00086E00E94BE0881E00E94C3083D98339A01
:1011B000109270057894089533983798089597B1F0
:1011C000907E8F71982B97B90895349A369A089526
:1011D00086B199278074907008951092700597B128
:1011E000907E8F71982B97B9349A369A3699FECFA4
:1011F00084B1282F332785B19927982F8827822BF0
:10120000932B08950E94ED0896958795969587955E
:10121000992708951F920F920FB60F9211248F9362
:101220008FEF809370058F910F900FBE0F901F90DE
:10123000189581E890E00E94BA03089584E890E050
:101240000E94BA03089599279F938F9389E890E0AD
:101250009F938F9381E08F930E94CE040F900F9005
:101260000F900F900F900895882319F08FE890E069
:1012700002C086E990E09F938F9381E08F930E9454
:10128000CE040F900F900F900895262F33273F9391
:101290002F9399279F938F938DE990E09F938F933E
:1012A00081E08F930E94CE048DB79EB707960FB64C
:1012B000F8949EBF0FBE8DBF0895109275051092D1
:1012C00071051092760510927305109272051092B6
:1012D000740508950F931F939C018B0190917405E1
:1012E0008FE0989FC0011124B901845A9D4F0E943C
:1012F0003E1380917405E82FFF27EE0FFF1FEC547B
:10130000FB4F118300838F5F809374051F910F91B2
:10131000089590930505809304050895CF93DF9376
:10132000C2ECD0E0FE018491882361F0FE01219699
:101330008491E0910405F09105050995FE018491E1
:101340008823A1F7DF91CF9108950F931F93CF9337
:10135000E0910405F09105058DE009950E948E0944
:10136000C091710507E715E0C150CF3F51F0E09102
:101370000405F0910505D8018D918D010995C150A5
:10138000B0F7CF911F910F9108959927009719F009
:10139000019761F00895809177058823D9F067E778
:1013A00075E087EC95E00E943E13089567EC75E0C8
:1013B00087E795E00E943E13E7E7F5E00190002003
:1013C000E9F73197E757F540E0937105E09376052B
:1013D0000E94A5090895CF93DF93C8EBD0E0FE01EA
:1013E0008491882349F0FE0121968491E0910405BF
:1013F000F09105050995F3CFC7E7D5E08091770512
:1014000009C0803249F0E0910405F0910505899109
:10141000099588818823A9F7E0910405F0910505D5
:101420008AE30995E0910405F091050580E20995AC
:10143000C6EAD0E0FE018491882349F0FE0121969E
:101440008491E0910405F09105050995F3CFE091B1
:101450000405F09105058DE00995E0910405F091F2
:1014600005058AE00995DF91CF910895FF920F93CA
:101470001F93CF93DF9300E0802F0E94C5098091D6
:101480007705803299F1882389F10F5FE02FFF27DC
:10149000E958FA4FE081E03211F0EE23B1F7002372
:1014A00071F424C0E12FFF27EE0FFF1FEC54FB4F18
:1014B00080819181909373058093720519C010E02B
:1014C000F09074051F1580F4CCE5D2E0802F9927A9
:1014D000AC0167E775E0CE010E944513892B11F33B
:1014E0001F5F2F961F1590F30E94EB090E948E0933
:1014F000DF91CF911F910F91FF9008951F93CF938C
:10150000182F20917505223009F045C099278234A3
:10151000910581F08334910524F48134910541F0E3
:1015200037C08334910551F08434910511F130C0F6
:1015300081E001C0822F0E94C5092AC090917605E2
:1015400080917105E0910405F09105059817F0F47C
:101550009F5F909376058BE10995E0910405F091EA
:1015600005058BE50995E0910405F091050583E4F7
:101570000EC080917605E0910405F0910505882361
:1015800029F081508093760588E001C087E00995B5
:1015900010927505EBC0213021F48B3511F482E0F7
:1015A000E3C010927505812F80528F3508F04DC031
:1015B00090917605809171059817B1F4E09104053A
:1015C000F0910505812F099580917605E82FFF2779
:1015D000E958FA4F10838F5F8093760580917105EB
:1015E0008F5F80937105C2C08F5F80937105C82F94
:1015F000981760F4A82FBB27A958BA4FFD0131975F
:1016000080818C93C150DF019C17C0F380917605D7
:10161000E82FFF27E958FA4F10838F5F80937605F4
:101620000E94A509C091760580917105C81708F040
:101630009DC0E0910405F091050588E00995CF5F14
:1016400080917105C817A8F391C01D3011F5E09184
:101650000405F0910505812F0995E0910405F091AD
:1016600005058AE0099580917105E82FFF27E95863
:10167000FA4F10828F5F80937105809176058F5F9E
:10168000809376050E94360A1092710510927605B5
:101690006DC0183009F063C080917605882309F485
:1016A00057C0909171058917E9F4E0910405F09114
:1016B0000505812F0995E0910405F091050580E26B
:1016C0000995E0910405F0910505812F0995809118
:1016D00071058150809371058091760581508093CA
:1016E000760544C0915090937105815080937605A2
:1016F000C82F891748F4E82FFF27E958FA4F81814E
:101700008193CF5FC917D8F30E94A509E091040522
:10171000F091050580E20995C09176052C2F3327BD
:10172000809171059927019628173907FCF4E091FB
:101730000405F091050588E00995CF5F2C2F33272C
:1017400080917105992701962817390784F30EC0F7
:10175000E0910405F091050587E0099507C01F3762
:1017600029F01B3119F481E080937505CF911F9109
:101770000895E0917205F0917305309739F009955D
:1017800010927305109272050E948E090895382FE9
:1017900090E080917705803239F49F5FE92FFF2731
:1017A000E958FA4F8081F7CF20E02317B0F403C047
:1017B000E03241F09F5FE92FFF27E958FA4FE081BF
:1017C000EE23B1F7E92FFF27E958FA4F80818032E5
:1017D00011F49F5FF7CF2F5FE8CF892F99278958A2
:1017E0009A4F0895CF93DF93CDB7DEB722970FB608
:1017F000F894DEBF0FBECDBF0E94C70B4AE050E099
:10180000BE016F5F7F4F0E943912DC01CB01BC012A
:10181000CD0122960FB6F894DEBF0FBECDBFDF918B
:10182000CF910895CF93DF93CDB7DEB722970FB650
:10183000F894DEBF0FBECDBF0E94C70B40E150E061
:10184000BE016F5F7F4F0E943912DC01CB01BC01EA
:10185000CD0122960FB6F894DEBF0FBECDBFDF914B
:10186000CF910895E199FECF9FBB8EBB6DBBE29AED
:10187000E19A0895EF92FF921F93CF93DF93CDB734
:10188000DEB721970FB6F894DEBF0FBECDBFEE24B2
:10189000FF240E941E0960E081E00E9445098DEE50
:1018A00091E00E94BA030E945D098AE892E00E94DA
:1018B00089096AE17DE084E890E00E946A096BE1B1
:1018C0007DE089E890E00E946A096FE17DE08EE8A2
:1018D00090E00E946A096CE57DE083E990E00E9457
:1018E0006A0968EA7DE086E990E00E946A096AEB8D
:1018F0007DE089E990E00E946A0964ED7DE08CE971
:1019000090E00E946A096DE77EE08FE990E00E9416
:101910006A0963E27DE083EA90E00E946A096EE072
:101920007EE086EA90E00E946A0968E17EE08AEA49
:1019300090E00E946A0967E27EE08EEA90E00E94F1
:101940006A0961E37EE082EB90E00E946A096EE63C
:101950007DE085EB90E00E946A096BE37EE088EB16
:1019600090E00E946A096AE47EE08BEB90E00E94BE
:101970006A0969E57EE08EEB90E00E946A096AE5FB
:101980007EE081EC90E00E946A098DE00E947E0A70
:101990008FEF8093670603C089810E947E0ACE0183
:1019A00001960E949302182F8823B1F70894E11C36
:1019B000F11C89EEE81683E0F80610F0EE24FF240F
:1019C000809106058823A1F06091790080E090E085
:1019D0000E94320C6091120581E090E00E94320C6E
:1019E0006091110582E090E00E94320C1093060590
:1019F0000E94B90B80916706882389F60E94CE0366
:101A00008DEF91E09F938F9381E08F930E94CE049E
:101A10000F900F900F9021960FB6F894DEBF0FBE77
:101A2000CDBFDF91CF911F91FF90EF90089510925D
:101A300067060895089580E00E94C308089581E034
:101A40000E94C3080895FF920F931F9329B386B392
:101A5000F3B200B399279F938F93822F99279F9377
:101A60008F938FE092E09F938F9311E01F930E94DA
:101A7000CE048DB79EB707960FB6F8949EBF0FBEE3
:101A80008DBF802F99279F938F938F2D99279F9399
:101A90008F9388E192E09F938F931F930E94CE04CF
:101AA0008DB79EB707960FB6F8949EBF0FBE8DBF39
:101AB0001F910F91FF90089589B399279F938F935A
:101AC00083E292E09F938F9381E08F930E94CE04F4
:101AD0000F900F900F900F900F9008951F9380918B
:101AE000190590911A059F938F9382E392E09F933B
:101AF0008F9311E01F930E94CE040F900F900F90D0
:101B00000F900F9080911505909116059F938F93DC
:101B100087E492E09F938F931F930E94CE040F90CF
:101B20000F900F900F900F908091080590910905EC
:101B30009F938F938CE592E09F938F931F930E94C6
:101B4000CE040F900F900F900F900F901F9108955B
:101B500086B399279F938F9381E792E09F938F930A
:101B600081E08F930E94CE040F900F900F900F9002
:101B70000F9008951F9383B399279F938F9382E8C3
:101B800092E09F938F9311E01F930E94CE04812FC8
:101B90000E94F20BDC01CB0185BB0F900F900F90E0
:101BA0000F900F901F9108951F930E94CE0380B352
:101BB00099279F938F9387E892E09F938F9311E0EB
:101BC0001F930E94CE04812F0E94F20BDC01CB01F7
:101BD00082BB0F900F900F900F900F901F91089560
:101BE00081E00E94F20BDC01CB018CBF08950895C7
:101BF000089581E00E94F20BDC01CB019C01832F50
:101C000099278BBD2ABD089581E00E94F20BDC016B
:101C1000CB0190937B0080937A00089581E00E942D
:101C2000F20BDC01CB019093760080937500089550
:101C300081E00E94F20BDC01CB018093740082E012
:101C40000E94F20BDC01CB0180937300089581E0C8
:101C50000E94F20BDC01CB01909378008093770017
:101C6000089581E00E94F20BDC01CB019093720099
:101C700080937100089581E00E94F20BDC01CB019A
:101C80008093610082E00E94F20BDC01CB01809323
:101C90006000089581E00E94F20BDC01CB0180938B
:101CA0005B0182E00E94F20BDC01CB0180935A01C0
:101CB000089508958FE790E08054904097FFFCCFFF
:101CC0008CE892E09F938F9381E08F930E94CE04E3
:101CD0000F900F900F908FE790E08054904097FF07
:101CE000FCCF8FE892E09F938F9381E08F930E94C7
:101CF000CE040F900F900F900895FF920F931F93B3
:101D0000CF93DF9320E030E0CBE3D5E08991999148
:101D10009F938F9389010F5F1F4F1F930F9382E94A
:101D200092E09F938F9391E0F92EFF920E94CE0450
:101D30008DB79EB707960FB6F8949EBF0FBE8DBFA6
:101D400098010830110510F38EE992E09F938F936C
:101D5000FF920E94CE040F900F900F90DF91CF91D1
:101D60001F910F91FF900895089580911B05909108
:101D70001C05009719F00197D1F035C081E090E083
:101D800090931C0580931B0583B3282F33272F7155
:101D900030708091190590911A05817E822B932BCA
:101DA00090931A0580931905AD9AAE981CC01092B5
:101DB0001C0510921B0583B3282F33272F71307019
:101DC0008091190590911A058F719C7F45E0220F33
:101DD000331F4A95E1F7822B932B90931A0580933A
:101DE0001905AD98AE9A8091190590911A0508953C
:101DF0009C01ECE5F1E0A2E9B1E08D919D918217A3
:101E0000930719F4808191810895329681E0E23937
:101E1000F8079CF380E89FEF089560E070E0209160
:101E2000770030917800280F391F33232CF461504C
:101E30007040245F3F4FF9CF2C3031052CF06F5F9D
:101E40007F4F2C503040F8CFC901820F931FFC0107
:101E5000EB53FF4F24913327322F22278A539F4F72
:101E6000FC018491280F311D40E050E084E090E0B7
:101E7000861B970B481759072CF4369527954F5F0B
:101E80005F4FF8CFC9010895959A80911D059091F3
:101E90001E05019690931E0580931D05883B9105B4
:101EA00088F110921E0510921D05809119059091E0
:101EB0001A0590931805809317050E94B50E9C0192
:101EC00090931A0580931905809117059091180534
:101ED00028173907B9F0C9010E94F80E909316052A
:101EE000809315052FEF8038920731F00E940D0F77
:101EF000909309058093080580EA9FE0909376000F
:101F00008093750080910A0590910B05209108053A
:101F100030910905820F931F90930B0580930A055A
:101F200020910F05309110052817390718F480917A
:101F3000730002C08091740083BD80910C05909164
:101F40000D05019690930D0580930C05209163007B
:101F50003091640028173907F8F410920D0510929B
:101F60000C058091750090917600825A9E4F909357
:101F700076008093750081549F4130F080EA9FE0A5
:101F80009093760080937500809175009091760013
:101F90009093100580930F0595980895282F332767
:101FA000E0911F05F09120052E1B3F0B80916000F2
:101FB00099276091210570912205689FA001699F72
:101FC000500D789F500D1124CA0146E095958795D4
:101FD0004A95E1F7281B390B3093240520932305FC
:101FE00080916100482F5527429FC001439F900D6B
:101FF000529F900D1124B6E095958795BA95E1F71B
:10200000860F971F9093220580932105489F90018A
:10201000499F300D589F300D1124C901A6E09595B8
:102020008795AA95E1F78E0F9F1F909320058093C7
:102030001F05F4E095958795FA95E1F78058992763
:102040000895CF93DF93CDB7DEB722970FB6F894FC
:10205000DEBF0FBECDBF809126058F5F8093260522
:10206000843040F010922605CE0101960E94131193
:102070008093250522960FB6F894DEBF0FBECDBF24
:10208000DF91CF91089589B78D7F89BF64E47FE0A8
:1020900087E00E9406069AE093BF8DE28CBF89B765
:1020A000826089BF89B78F7E89BF89B78F7789BFE3
:1020B00089E785BD93BD0895CFE5D8E0DEBFCDBFEC
:1020C0000E94660260E071EE80E090E00E943602BD
:1020D0008AE892E00E9462030E94CE080E941909D9
:1020E00081EA92E09F938F9381E08F930E94CE04C8
:1020F0001ABA1BBA17BA9FEF98BB80E684BB8FE170
:1021000085BB91BB12BA969A0E9443100E943A0C6A
:102110000F900F900F9080E090E00C9405140895BC
:10212000089508950895E199FECF9FBB8EBBE09A74
:102130008DB399270895BF92CF92DF92EF92FF92CD
:102140000F931F93CF93DF93EE24FF24670100E0EA
:1021500010E0E601CE010E94931099279F938F9380
:102160008EEC92E09F938F9351E0B52EBF920E9428
:10217000CE040F900F900F900F900F900F5F1F4F96
:1021800021960032110534F382ED92E09F938F93F4
:10219000BF920E94CE040F900F900F900894E11C04
:1021A000F11C80E290E0C80ED91E1E141F047CF6BC
:1021B000DF91CF911F910F91FF90EF90DF90CF9023
:1021C000BF9008956091C4007091C500AB01442791
:1021D000550F441F55279B012070307424E0329F17
:1021E000212D33271124CB0180709071892F9927DD
:1021F00082958F7042275327482759279B01220F2A
:10220000331F242B352B3093C5002093C4008091BD
:10221000C6009091C700842B952B9093C7008093A4
:10222000C600C9010895FC0184B1682F772785B1E4
:10223000482F55279A012370307080914B059927BC
:10224000009719F00197A1F160C080914C058F5F54
:1022500080934C05909159018917E0F4322F222781
:10226000330F330F660F771F660F771F260F371F49
:1022700030932A052093290541FF03C080E098E0B0
:1022800002C080E098EF2827392730932A05209351
:1022900029053BC010924C0580914D058F5F8770DA
:1022A00080934D05805C87B981E080934B052DC0FC
:1022B00010924B05522F4427460F571F51834083DE
:1022C00084E487B980914D05682F7727CB01860F6D
:1022D000971FFC01E55CFA4F51834083FC01E55DEB
:1022E000FA4F808191819A01281B390B37FF03C077
:1022F000309521953F4F809158019927281739072C
:1023000014F051834083CB01089586EC86B983E6AF
:1023100090E00895EF92FF920F931F93CF93DF9376
:102320008091540790915507FC0136E0F695E795AA
:102330003A95E1F7EE0FFF1FEA5AF84FC081D181BD
:102340002091520730915307280F391F30935507BA
:102350002093540740E12030340728F03F70309339
:10236000550720935407C058DF4F80914F058F5F6A
:1023700080934F05843008F449C010924F05809136
:102380005B01082F112760914E05A62FBB27FD0189
:10239000FF96EF73F070EE0FFF1FEA5AF84F80813F
:1023A0009181089F9001099F300D189F300D1124D5
:1023B00080915A01482F5527FD01EA0FFB1FEA5A69
:1023C000F84F80819181489F7001499FF00C589F80
:1023D000F00C11242E0D3F1D1196AF73B070AA0F93
:1023E000BB1FAA5AB84F8D919C91089FA001099FCD
:1023F000500D189F500D1124240F351F232F332704
:10240000318320836F5F6F7360934E058C2F992704
:10241000DF91CF911F910F91FF90EF90089510924F
:10242000550710925407E2EDF6E0A6E5B7E01D92DD
:102430001D921192119287E0E035F807C1F3BCF3C9
:1024400089E190E090935307809352078CE090E0ED
:1024500090935507809354078FE090E0909357072F
:102460008093560788E090E090935907809358072F
:102470000895A0E0B0E0EFE3F2E10C94D0138C01FA
:102480002B01EA01EE246115710519F0FB0191831E
:102490008083209749F0CE010297839728F060E06F
:1024A00070E080E090E0E5C0F801F1908F018F2DA1
:1024B00099270E94C313892BB9F7FDE2FF1619F47F
:1024C00041E0E42E03C0FBE2FF1619F4F801F1909D
:1024D0008F01209719F0C031D10591F4F0E3FF1678
:1024E00079F4F8018081883711F0883549F4F801D2
:1024F000F1800E5F1F4FC0E1D0E0F2E0EF2A0AC08A
:10250000209741F480E3F81619F4C8E0D0E002C047
:10251000CAE0D0E0C830D105E9F0C930D10524F4D3
:10252000C230D105E9F022C0CA30D10521F0C03156
:10253000D10551F01BC03CECA32E3CECB32E3CEC7F
:10254000C32E3CE0D32E1FC0A12CB12CC12C28E0FF
:10255000D22E19C0A12CB12CC12C90E1D92E13C0C0
:10256000A12CB12CC12C80E4D82E0DC09E01442793
:1025700037FD4095542F60E070E080E090E80E94C5
:10258000861359016A0120E030E040E050E060E04D
:102590003E01882477FC8094982C8F2D80538A30BC
:1025A00010F4F82E0DC08F2D81548A3118F4E9EC07
:1025B000FE0E06C08F2D81568A3148F5F9EAFF0ECE
:1025C0008F2D99278C179D0714F567FD1CC0A21647
:1025D000B306C406D506A0F0CA01B901A40193014F
:1025E0000E9453139B01AC012F0D311D411D511D44
:1025F000213080E0380780E0480780E8580710F075
:102600006FEF01C061E0F801F1908F01C6CF411476
:10261000510461F0662319F00150104004C0E1FE3E
:1026200005C002501040F201118300838E2D9927BE
:1026300067FF07C080FF11C020E030E040E050E8B5
:1026400010C080FF08C050954095309521953F4FB0
:102650004F4F5F4F0CC057FF0AC02FEF3FEF4FEFB8
:102660005FE782E290E09093D7078093D607CA0194
:10267000B901E0E1CDB7DEB70C94EC13FB01DC014E
:1026800001900D920020E1F70895FB01DC0141501B
:10269000504030F08D910190801919F40020B9F765
:1026A000881B990B0895629FD001739FF001829F50
:1026B000E00DF11D649FE00DF11D929FF00D839FD1
:1026C000F00D749FF00D659FF00D9927729FB00D6E
:1026D000E11DF91F639FB00DE11DF91FBD01CF0181
:1026E00011240895AA1BBB1B51E107C0AA1FBB1FE1
:1026F000A617B70710F0A61BB70B881F991F5A958E
:10270000A9F780959095BC01CD010895A1E21A2EFC
:10271000AA1BBB1BFD010DC0AA1FBB1FEE1FFF1F85
:10272000A217B307E407F50720F0A21BB30BE40BD5
:10273000F50B661F771F881F991F1A9469F760951C
:102740007095809590959B01AC01BD01CF010895D6
:1027500097FB092E05260ED057FD04D0D7DF0AD0EF
:10276000001C38F450954095309521953F4F4F4FC0
:102770005F4F0895F6F790958095709561957F4F1E
:102780008F4F9F4F0895911106C0803219F08950E4
:102790008550D0F708959927882708952F923F9262
:1027A0004F925F926F927F928F929F92AF92BF9261
:1027B000CF92DF92EF92FF920F931F93CF93DF930D
:1027C000CDB7DEB7CA1BDB0B0FB6F894DEBF0FBE6A
:1027D000CDBF09942A88398848885F846E847D84B7
:1027E0008C849B84AA84B984C884DF80EE80FD80B9
:1027F0000C811B81AA81B981CE0FD11D0FB6F8942F
:0C280000DEBF0FBECDBFED010895FFCF7D
:10280C000A3C63BC02F00AC012901AA82FC05D608B
:10281C006D2E00FF0AA00FC4FFFFE8030A00FF00A3
:10282C000000FF0068656C7000617265660061767F
:10283C00636300706100706200706300706400611B
:10284C0064630070700070776D00706C68006F6668
:10285C006600616D006B64007376006162007362E8
:10286C000064730001000100400118010A01FC0022
:10287C00F200E800260134010C00070007000700F5
:10288C00050005000600000000000400050007001C
:10289C00090000000300050007000A000000020008
:1028AC0003000500070008000B00000002000300F5
:1028BC000500070008000A000000020004000500E3
:1028CC00070009000B0000000200030005000600D1
:1028DC0008000900000002000400060008000A00BD
:1028EC0000000100020003000400050006000700C0
:1028FC00080009000A000B00140A32040C0009003D
:10290C00050002000B0007000400000006000A008E
:10291C000100030008001800150011000E0017003C
:10292C00130010000C00120016000D000F00140014
:10293C000000BF013F037F02FF00BF037F03FF02C4
:10294C00FF013F02BF027F017F003F00ED03F9034F
:10295C00F303E703FD03FB03F703EF03F103F503B5
:08296C00EB03E303E1030000AB
:00000001FF
